S01A0000417454696E795F616C61726D5F636C6F636B2E73726563DA
S113000014C019C018C017C016C015C014C013C03E
S113001012C011C010C00FC00EC00DC00CC00BC068
S11300200AC009C008C007C006C011241FBECFED16
S1130030CDBF80D089C0E4CFCF93C2E362D0C1509A
S1130040E9F7CF910895CF93C62F843038F48230E6
S113005048F4882371F0813049F00CC0843051F4A5
S1130060939808C04F73833009F4405C842F8068F0
S113007024D0939A929A929A98B39F708C2F807FEF
S1130080982B98BB98B39F70892B88BB92989298B1
S113009038D087B3803F79F4929A929A88B3C29504
S11300A0C07F8F708C2B88BB88B38F70C82BC8BB64
S11300B09298929826D0CF91089540E0682F84E0DA
S11300C0C2DF08958FEF87BB8B9A8A9A88BB939A75
S11300D0929AB2DFB1DFB0DF80E3EFDFADDF80E320
S11300E0ECDF0FD080E3E9DF88E2E7DF87B3807FCE
S11300F087BB8CE0E2DF86E0E0DF82E0DEDF9CDFCE
S11301000895CF93DF931F92CDB7DD2784E48983CD
S113011089819FEF980F9983882341F08981898190
S113012089819FEF980F99838111F8CF0F90DF9108
S1130130CF9108958FEF87BB8AEA88BBC3DF40E085
S10F014061E480E080DFFFCFF894FFCF83
S9030000FC
